:020000020000FC
:100000000DC045C0000000006CC06FC078C000008B
:1000100000000000626B6F34303774310FED0DBF9C
:1000200000E008BB0CEF07BB08E702BB00E001BB28
:1000300002E003BF02E00EBD772788279927D8D1B9
:1000400004E6B02EC4D0C3D0AED002E3302E0BEF06
:10005000202E00E0C02ED02E02EC08BF09BF7894FD
:1000600003E005BF00E40BBF2AE083FFFECF092DAC
:100070001A2D877F0C541440B8F72A95B1F7F894DD
:1000800092D091D078940EE100936D00D2C11FB64A
:1000900044274BBF45B740FF09C0829B1EC042E0CA
:1000A00045BF4CB55DB5742E852E17C0829915C01D
:1000B00043E045BF83FD11C04CB55DB547195809F4
:1000C000942EA52E483968E0560738F4403263E094
:1000D000560718F0886044E6B42E50E45BBF1FBE9C
:1000E00018951FB67E7F1FBE18951FB67068EE204C
:1000F00009F0EA94BB2009F0BA941FBE18951FB608
:1001000076FD2BC040B340937000422D562D5417FE
:1001100030F43A9459F452E3352E4A9506C031F042
:100120003A9421F458E2352E4395242E706474FFDE
:1001300008C094FF03C0839B72609F7E81FFC698B6
:1001400007C075FF03C081FFC79802C081FFC59833
:10015000422D4C59409542BF22C0422D42BF7F7B69
:1001600074FF03C080FFC69A07C075FF03C080FFFD
:10017000C79A02C080FFC59A4D3918F482608E7FFD
:1001800007C04B3F18F08D7F816002C08D7F8E7F4E
:1001900086FF05C0C59B03C0459B74608F7B93FDA4
:1001A00081601FBE189510E8002702BFC49AC79A45
:1001B00002B70032E9F7C498C79828E0002702BFC9
:1001C00002B70F3FE9F72A95C9F71A9569F710E8C2
:1001D00028E0002702BF02B70F3FE9F72A95C9F7C9
:1001E0001A95B1F7089530E03BBF000000000CB550
:1001F0001DB508958F7E83FF14C0092D1A2D877FAA
:100200000C54144010F400271127169507951695E5
:10021000079516950795202F0456104008F024E600
:10022000F22F08958F7708958F7D77FF17C07F771E
:1002300072FF06C07B7F4C2D433090F4C39403C003
:10024000CC2009F0CA9471FF06C07D7F4D2D443645
:1002500028F4D39403C0DD2009F0DA94A6D00895E1
:10026000F894DCCEC0DF00936000109361000C0FA7
:100270001D1F32E839BF1BBD0ABD716032EC39BFAA
:1002800030E43BBF0091640010916500E09166008E
:10029000E69517950795E6951795079520916400C3
:1002A00030916500E0916600201B310BE040009129
:1002B000600010916100C0916200D09163000093D2
:1002C0006200109363000C1B1D0B200F311F10E008
:1002D000E11F2093640030936500E0936600089569
:1002E000C0916700D0916800BDDFE69537952795EE
:1002F000E69537952795E69537952795E6953795B1
:10030000279520936700309368002093690030930D
:100310006A00089570FDFECF7160DFE1C0E463DF25
:100320000C0F1D1F32E839BF1BBD0ABD32EC39BFAF
:1003300030E43BBF0895716056DFC0916900D091F1
:100340006A000C0F1D1F22E829BF1BBD0ABD22EC4D
:1003500029BF30E43BBF84FD4DDF85FD65DF70FDC7
:10036000FECF0895C0916B00D0916C007BDF56D01A
:1003700055D00895C0916B00D0916C00DF3168F0CA
:100380000C2F1D2F16950795169507951695079511
:1003900016950795C01BD10B02C0C0E8DBEBC093DC
:1003A0006B00D0936C00946008950F2F0D1908F422
:1003B00004E095FF05C01AE00117B8F0012F15C041
:1003C00010916500103438F09160926019E10117C6
:1003D00060F0012F0AC0103238F09E7F926012E365
:1003E000011718F0012F01C09C7F0095602E089521
:1003F000F4E00BEF202E602E00E008BB02E3302E6D
:10040000C0E8DBEBC0936B00D0936C008160977FFA
:100410009062089504E00A95F1F7089576FDFECF05
:1004200076FFFECF00917000089508950895089515
:100430000895DEDFFDDFDEDEF530E8F30AEF202E83
:10044000602E00EC09BF00007F7D7061C49A81FDC1
:1004500002C076FD03C0C79880FFC69A02EC09BFB0
:100460009B7F00E000936E0004E6E02E7BDF70FDD2
:1004700002C080DF0CC0D2DFD8DF05FDF8CF70FDF1
:1004800002C078DF04C0CADFD0DF05FFF8CFF0D0AC
:1004900069DF70FD02C06EDF0CC0C0DFC7DF04FF84
:1004A000F8CF70FD02C066DF04C0B8DFBFDF04FD17
:1004B000F8CFE2D09FDE56DF70FD02C05BDF0CC0DC
:1004C000ADDFB5DF06FDF8CF70FD02C053DF04C01D
:1004D000A5DFADDF06FFF8CFDED0A4DE43DF70FD81
:1004E00002C048DF0CC09ADFA0DF05FFF8CF70FD27
:1004F00002C040DF04C092DF98DF05FDF8CFCFD007
:1005000031DF70FD02C036DF0CC088DF8FDF04FDF5
:10051000F8CF70FD02C02EDF04C080DF87DF04FF4C
:10052000F8CFCCD081DE00916600002341F4009129
:100530006500043120F410916F00139501C011275C
:1005400010936F000FDF70FD02C014DF0CC066DF78
:100550006EDF06FFF8CF70FD02C00CDF04C05EDF67
:1005600066DF06FDF8CFAED0022D0B3F08F061CF5D
:10057000BB2009F47AC0EE2009F477C000916F0027
:10058000043150F400916E0092FD00270395009312
:100590006E009B7F023330F00FEFF02EA1DEBCDE49
:1005A0009F7D02C0DFDE63CF70FD01C042CF859B1F
:1005B000FBCF30DF859BF8CFBEDE5AD091DEAADEBE
:1005C000906170FD01C035CF8499FBCF23DF849902
:1005D000F8CF8061B0DE9F7E4FD082DE9BDE70FD63
:1005E00001C027CF869BFBCF15DF869BF8CF8068A5
:1005F000A2DE51D075DE8EDE806470FD01C019CFA1
:100600008599FBCF07DF8599F8CF95DE8F7B47D0A3
:1006100067DE80DE70FD01C00CCF849BFBCFFADE6D
:10062000849BF8CF806287DE49D05ADE73DE70FD8E
:1006300001C0FFCE8699FBCFEDDE8699F8CF7BDE39
:1006400041D04EDE67DEBB2081F0022D0B3F08F06B
:10065000F0CE977FFF2041F0FA9429F00F2D013062
:1006600011F0023009F498609FCFF894C1DED6CC27
:10067000C49880FFC39A089500EC09BF00007F7DF5
:100680007F7E81FD02C076FD03C0C69880FFC59ABB
:1006900002EC09BF0895C39880FFC29A089500EC48
:1006A00009BF000070627F7E81FD02C076FD03C03D
:1006B000C59880FFC79A02EC09BF0895C29880FFD1
:1006C000C49A089500EC09BF00007F7D706181FD30
:1006D00002C076FD03C0C79880FFC69A02EC09BF2E
:0206E00008957B
:00000001FF
